:0200000480007A
:100000006F000005732F2034930F80006308FF03F7
:10001000930F90006304FF03930FB0006300FF038E
:10002000130F000063040F0067000F00732F2034CC
:1000300063540F006F00400093E19153171F0000BD
:1000400023223FFC171F000023200FFC6FF01FFF2F
:100050009300000013010000930100001302000050
:100060009302000013030000930300001304000038
:100070009304000013050000930500001306000020
:100080009306000013070000930700001308000008
:10009000930800001309000093090000130A0000F0
:1000A000930A0000130B0000930B0000130C0000D8
:1000B000930C0000130D0000930D0000130E0000C0
:1000C000930E0000130F0000930F0000732540F102
:1000D0006310050097020000938202017390523072
:1000E000735044749702000093820201739052305F
:1000F00073500018970200009382420273905230AE
:100100009B021000939252039382F2FF7390023B82
:100110009302F0017390023A73504030970200004E
:1001200093824201739052307350203073503030BC
:100130009301000097020000938202ED7390523009
:10014000130510001315F501635C05000F00F00F97
:10015000930110009308D005130500007300000000
:1001600093020000638A020073905210B7B200003D
:100170009B829210739022307350003097020000DF
:100180009382420173901234732540F17300203042
:1001900093012000930000001301000033872040EA
:1001A00093030000631E774A930130009300100010
:1001B0001301100033872040930300006312774A35
:1001C00093014000930030001301700033872040FA
:1001D0009303C0FF6316774893015000930000001B
:1001E0003781FFFF33872040B7830000631A7746CB
:1001F00093016000B70000801301000033872040A6
:10020000B7030080631E774493017000B70000803D
:100210003781FFFF33872040B78300806312774424
:100220009301800093000000378100001B01F1FF63
:1002300033872040B783FFFF9B831300631277420D
:1002400093019000B70000809B80F0FF1301000035
:1002500033872040B70300809B83F3FF631277400E
:100260009301A000B70000809B80F0FF3781000061
:100270001B01F1FF33872040B783FF7F6312773E76
:100280009301B000B7000080378100001B01F1FF2F
:1002900033872040B703FFFF9B83F3FF9393F30063
:1002A00093831300631E773A9301C000B700008068
:1002B0009B80F0FF3781FFFF33872040B7030100A9
:1002C0009B8313009393F3009383F3FF631A7738B0
:1002D0009301D000930000001301F0FF338720400A
:1002E00093031000631E77369301E0009300F0FF44
:1002F00013011000338720409303E0FF6312773629
:100300009301F0009300F0FF1301F0FF33872040CA
:100310009303000063167734930100019300D0002B
:100320001301B000B380204093032000639A703221
:10033000930110019300E0001301B00033812040CD
:1003400093033000631E7130930120019300D000AD
:10035000B380104093030000639470309301300128
:10036000130200009300D0001301B0003387204037
:10037000130307001302120093022000E31452FE3D
:1003800093032000631E732C9301400113020000AD
:100390009300E0001301B0003387204013000000F9
:1003A000130307001302120093022000E31252FE0F
:1003B000930330006316732A930150011302000067
:1003C0009300F0001301B0003387204013000000B9
:1003D0001300000013030700130212009302200011
:1003E000E31052FE93034000631C732693016001E7
:1003F000130200009300D0001301B00033872040A7
:100400001302120093022000E31652FE9303200011
:100410006318772493017001130200009300E00039
:100420001301B000130000003387204013021200B4
:1004300093022000E31452FE9303300063127722EC
:1004400093018001130200009300F0001301B0003B
:100450001300000013000000338720401302120035
:1004600093022000E31252FE93034000631A771EAA
:1004700093019001130200009300D00013000000CC
:100480001301B000338720401302120093022000B2
:10049000E31452FE930320006314771C9301A00120
:1004A000130200009300E000130000001301B000ED
:1004B0001300000033872040130212009302200033
:1004C000E31252FE93033000631C77189301B001CE
:1004D000130200009300F00013000000130000005E
:1004E0001301B00033872040130212009302200052
:1004F000E31252FE93034000631477169301C00188
:10050000130200001301B0009300D0003387204095
:100510001302120093022000E31652FE9303200000
:10052000631077149301D001130200001301B0008F
:100530009300E000130000003387204013021200F4
:1005400093022000E31452FE93033000631A7710E5
:100550009301E001130200001301B0009300F000CA
:100560001300000013000000338720401302120024
:1005700093022000E31252FE930340006312770EB1
:100580009301F001130200001301B00013000000FA
:100590009300D00033872040130212009302200002
:1005A000E31452FE93032000631C770A93010002B8
:1005B000130200001301B000130000009300E000DC
:1005C0001300000033872040130212009302200022
:1005D000E31252FE93033000631477089301100274
:1005E000130200001301B00013000000130000000C
:1005F0009300F00033872040130212009302200082
:10060000E31252FE93034000631C7704930120021F
:10061000930010FF330110409303F0006312710444
:1006200093013002930000023381004093030002E3
:100630006318710293014002B3000040930300006D
:100640006390700293015002930000011301E001D6
:100650003380204093030000631470006310300265
:100660000F00F00F638001009391110093E11100DE
:100670009308D00513850100730000000F00F00FF0
:10068000930110009308D0051305000073000000CB
:10069000731000C000000000000000000000000017
:1006A000000000000000000000000000000000004A
:0C06B0000000000000000000000000003E
:1010000000000000000000000000000000000000E0
:1010100000000000000000000000000000000000D0
:1010200000000000000000000000000000000000C0
:1010300000000000000000000000000000000000B0
:081040000000000000000000A8
:040000058000000077
:00000001FF
